 FARCmds

 Timestamp is 537255bb (Tue May 13 21:26:19 2014)

 Preferred load address is 0000000180000000

 Start         Length     Name                   Class
 0001:00000000 00000168H .idata$5                CODE
 0001:00000170 00000616H .rdata                  CODE
 0001:00000790 00005335H .text                   CODE
 0001:00005ac8 000003ecH .xdata                  CODE
 0001:00005eb4 00000028H .idata$2                CODE
 0001:00005edc 00000014H .idata$3                CODE
 0001:00005ef0 00000168H .idata$4                CODE
 0001:00006058 00000328H .idata$6                CODE
 0001:00006380 000000a5H .edata                  CODE
 0002:00000000 00000058H .data                   DATA
 0002:00000060 00004340H .bss                    DATA
 0003:00000000 0000033cH .pdata                  DATA
 0004:00000000 00000058H .rsrc$01                DATA
 0004:00000060 00000378H .rsrc$02                DATA

  Address         Publics by Value              Rva+Base               Lib:Object

 0000:00000000       ___safe_se_handler_table   0000000000000000     <absolute>
 0000:00000000       ___safe_se_handler_count   0000000000000000     <absolute>
 0000:00000000       __ImageBase                0000000180000000     <linker-defined>
 0001:00000000       __imp_RegQueryValueExW     0000000180001000     advapi32:ADVAPI32.dll
 0001:00000008       __imp_RegCloseKey          0000000180001008     advapi32:ADVAPI32.dll
 0001:00000010       __imp_RegOpenKeyExW        0000000180001010     advapi32:ADVAPI32.dll
 0001:00000018       \177ADVAPI32_NULL_THUNK_DATA 0000000180001018     advapi32:ADVAPI32.dll
 0001:00000020       __imp_lstrcatW             0000000180001020     kernel32:KERNEL32.dll
 0001:00000028       __imp_GetModuleFileNameW   0000000180001028     kernel32:KERNEL32.dll
 0001:00000030       __imp_GetProcAddress       0000000180001030     kernel32:KERNEL32.dll
 0001:00000038       __imp_GetModuleHandleW     0000000180001038     kernel32:KERNEL32.dll
 0001:00000040       __imp_CloseHandle          0000000180001040     kernel32:KERNEL32.dll
 0001:00000048       __imp_RemoveDirectoryW     0000000180001048     kernel32:KERNEL32.dll
 0001:00000050       __imp_DeleteFileW          0000000180001050     kernel32:KERNEL32.dll
 0001:00000058       __imp_GetFileSize          0000000180001058     kernel32:KERNEL32.dll
 0001:00000060       __imp_CreateFileW          0000000180001060     kernel32:KERNEL32.dll
 0001:00000068       __imp_lstrcpyW             0000000180001068     kernel32:KERNEL32.dll
 0001:00000070       __imp_WriteConsoleW        0000000180001070     kernel32:KERNEL32.dll
 0001:00000078       __imp_ReadFile             0000000180001078     kernel32:KERNEL32.dll
 0001:00000080       __imp_Sleep                0000000180001080     kernel32:KERNEL32.dll
 0001:00000088       __imp_GetTempFileNameW     0000000180001088     kernel32:KERNEL32.dll
 0001:00000090       __imp_CreateDirectoryW     0000000180001090     kernel32:KERNEL32.dll
 0001:00000098       __imp_MultiByteToWideChar  0000000180001098     kernel32:KERNEL32.dll
 0001:000000a0       __imp_GetACP               00000001800010a0     kernel32:KERNEL32.dll
 0001:000000a8       __imp_GetConsoleOutputCP   00000001800010a8     kernel32:KERNEL32.dll
 0001:000000b0       __imp_ExpandEnvironmentStringsW 00000001800010b0     kernel32:KERNEL32.dll
 0001:000000b8       __imp_WaitForSingleObject  00000001800010b8     kernel32:KERNEL32.dll
 0001:000000c0       __imp_CreateThread         00000001800010c0     kernel32:KERNEL32.dll
 0001:000000c8       __imp_CreateProcessW       00000001800010c8     kernel32:KERNEL32.dll
 0001:000000d0       __imp_SetConsoleTitleW     00000001800010d0     kernel32:KERNEL32.dll
 0001:000000d8       __imp_GetConsoleTitleW     00000001800010d8     kernel32:KERNEL32.dll
 0001:000000e0       __imp_SetCurrentDirectoryW 00000001800010e0     kernel32:KERNEL32.dll
 0001:000000e8       __imp_GetCurrentDirectoryW 00000001800010e8     kernel32:KERNEL32.dll
 0001:000000f0       __imp_SetConsoleMode       00000001800010f0     kernel32:KERNEL32.dll
 0001:000000f8       __imp_SetConsoleCursorPosition 00000001800010f8     kernel32:KERNEL32.dll
 0001:00000100       __imp_GetConsoleScreenBufferInfo 0000000180001100     kernel32:KERNEL32.dll
 0001:00000108       __imp_GetConsoleMode       0000000180001108     kernel32:KERNEL32.dll
 0001:00000110       __imp_GetStdHandle         0000000180001110     kernel32:KERNEL32.dll
 0001:00000118       __imp_SearchPathW          0000000180001118     kernel32:KERNEL32.dll
 0001:00000120       __imp_GetEnvironmentVariableW 0000000180001120     kernel32:KERNEL32.dll
 0001:00000128       __imp_HeapFree             0000000180001128     kernel32:KERNEL32.dll
 0001:00000130       __imp_GetProcessHeap       0000000180001130     kernel32:KERNEL32.dll
 0001:00000138       __imp_HeapAlloc            0000000180001138     kernel32:KERNEL32.dll
 0001:00000140       __imp_lstrlenW             0000000180001140     kernel32:KERNEL32.dll
 0001:00000148       __imp_GetFileAttributesW   0000000180001148     kernel32:KERNEL32.dll
 0001:00000150       __imp_ScrollConsoleScreenBufferW 0000000180001150     kernel32:KERNEL32.dll
 0001:00000158       __imp_lstrcpynW            0000000180001158     kernel32:KERNEL32.dll
 0001:00000160       \177KERNEL32_NULL_THUNK_DATA 0000000180001160     kernel32:KERNEL32.dll
 0001:00000170       ??_C@_1BI@BKNCFIOG@?$AAM?$AAa?$AAx?$AAD?$AAa?$AAt?$AAa?$AAS?$AAi?$AAz?$AAe?$AA?$AA@ 0000000180001170     FARCmds.obj
 0001:00000188       ??_C@_1BK@LOJIPNKK@?$AAE?$AAd?$AAi?$AAt?$AAN?$AAe?$AAw?$AAF?$AAi?$AAl?$AAe?$AAs?$AA?$AA@ 0000000180001188     FARCmds.obj
 0001:000001a8       ??_C@_1BM@BMDAMABJ@?$AAV?$AAi?$AAe?$AAw?$AAZ?$AAe?$AAr?$AAo?$AAF?$AAi?$AAl?$AAe?$AAs?$AA?$AA@ 00000001800011a8     FARCmds.obj
 0001:000001c8       ??_C@_1BE@EKEFMMPP@?$AAC?$AAa?$AAt?$AAc?$AAh?$AAM?$AAo?$AAd?$AAe?$AA?$AA@ 00000001800011c8     FARCmds.obj
 0001:000001e0       ??_C@_1BM@IEHCKIMD@?$AAS?$AAh?$AAo?$AAw?$AAC?$AAm?$AAd?$AAO?$AAu?$AAt?$AAp?$AAu?$AAt?$AA?$AA@ 00000001800011e0     FARCmds.obj
 0001:00000200       ??_C@_1BE@KBOCGMKN@?$AAS?$AAe?$AAp?$AAa?$AAr?$AAa?$AAt?$AAo?$AAr?$AA?$AA@ 0000000180001200     FARCmds.obj
 0001:00000218       ??_C@_1BM@FDPIJPAH@?$AAA?$AAd?$AAd?$AA2?$AAD?$AAi?$AAs?$AAk?$AAs?$AAM?$AAe?$AAn?$AAu?$AA?$AA@ 0000000180001218     FARCmds.obj
 0001:00000238       ??_C@_1BK@EJEHIDJM@?$AAA?$AAd?$AAd?$AA2?$AAP?$AAl?$AAu?$AAg?$AAM?$AAe?$AAn?$AAu?$AA?$AA@ 0000000180001238     FARCmds.obj
 0001:00000258       MainGuid                   0000000180001258     FARCmds.obj
 0001:00000268       SameFolderMenuGuid         0000000180001268     FARCmds.obj
 0001:00000278       ConfigMenuGuid             0000000180001278     FARCmds.obj
 0001:00000288       DialogGuid                 0000000180001288     FARCmds.obj
 0001:00000298       ??_C@_13HOIJIPNN@?$AA?5?$AA?$AA@ 0000000180001298     FARCmds.obj
 0001:0000029c       ??_C@_15BNIPFGCG@?$AA$?$AA?$CK?$AA?$AA@ 000000018000129c     FARCmds.obj
 0001:000002a8       ??_C@_1BE@EKCMLKPN@?$AA?$CF?$AAC?$AAO?$AAM?$AAS?$AAP?$AAE?$AAC?$AA?$CF?$AA?$AA@ 00000001800012a8     FARCmds.obj
 0001:000002c0       ??_C@_0BB@BNALAELI@GetConsoleAliasW?$AA@ 00000001800012c0     FARCmds.obj
 0001:000002d8       ??_C@_1BC@GDMECMAK@?$AAk?$AAe?$AAr?$AAn?$AAe?$AAl?$AA3?$AA2?$AA?$AA@ 00000001800012d8     FARCmds.obj
 0001:000002ec       ??_C@_13FPGAJAPJ@?$AA?2?$AA?$AA@ 00000001800012ec     FARCmds.obj
 0001:000002f0       ??_C@_1BE@BNONMOPA@?$AA?2?$AA?2?$AA?4?$AA?2?$AAc?$AAd?$AAr?$AAo?$AAm?$AA?$AA@ 00000001800012f0     FARCmds.obj
 0001:00000308       ??_C@_1CE@JKDBMIKG@?$AA?2?$AA?2?$AA?4?$AA?2?$AAP?$AAh?$AAy?$AAs?$AAi?$AAc?$AAa?$AAl?$AAD?$AAr?$AAi?$AAv?$AAe?$AA?$AA@ 0000000180001308     FARCmds.obj
 0001:00000330       ??_C@_19BKJMDJK@?$AA?2?$AA?2?$AA?4?$AA?2?$AA?$AA@ 0000000180001330     FARCmds.obj
 0001:00000340       ??_C@_17IJMNDCL@?$AA?$CF?$AAl?$AAu?$AA?$AA@ 0000000180001340     FARCmds.obj
 0001:00000348       ??_C@_1BA@EIPEFBMB@?$AA?$CF?$AAl?$AAu?$AA?1?$AA?$CF?$AAl?$AAu?$AA?$AA@ 0000000180001348     FARCmds.obj
 0001:00000360       ??_C@_19LJDFFCJJ@?$AA?$CF?$AAs?$AA?$CF?$AAs?$AA?$AA@ 0000000180001360     FARCmds.obj
 0001:0000036c       ??_C@_13NEIAEHFG@?$AA?$CC?$AA?$AA@ 000000018000136c     FARCmds.obj
 0001:00000370       ??_C@_1BM@MDBPDFDA@?$AA?$CF?$AAC?$AAO?$AAM?$AAS?$AAP?$AAE?$AAC?$AA?$CF?$AA?5?$AA?1?$AAc?$AA?5?$AA?$AA@ 0000000180001370     FARCmds.obj
 0001:0000038c       ??_C@_15GBHPEJPD@?$AA?1?$AAS?$AA?$AA@ 000000018000138c     FARCmds.obj
 0001:00000394       ??_C@_15MDAMMGLB@?$AA?1?$AAN?$AA?$AA@ 0000000180001394     FARCmds.obj
 0001:000003a0       ??_C@_19JMGCACDF@?$AA?1?$AAM?$AAS?$AAG?$AA?$AA@ 00000001800013a0     FARCmds.obj
 0001:000003ac       ??_C@_11LOCGONAA@?$AA?$AA@ 00000001800013ac     FARCmds.obj
 0001:000003b0       ??_C@_1GO@MIKMNHBD@?$AAS?$AAO?$AAF?$AAT?$AAW?$AAA?$AAR?$AAE?$AA?2?$AAM?$AAi?$AAc?$AAr?$AAo?$AAs?$AAo?$AAf?$AAt?$AA?2?$AAW?$AAi?$AAn?$AAd?$AAo?$AAw?$AAs?$AA?2?$AAC?$AAu?$AAr?$AAr?$AAe@ 00000001800013b0     FARCmds.obj
 0001:00000420       ??_C@_13PJJBFPED@?$AA?$DL?$AA?$AA@ 0000000180001420     FARCmds.obj
 0001:00000428       ??_C@_17IBNHEMGL@?$AA?$CF?$AAs?$AA?$DL?$AA?$AA@ 0000000180001428     FARCmds.obj
 0001:00000430       ??_C@_1BA@IBNPAI@?$AAF?$AAA?$AAR?$AAH?$AAO?$AAM?$AAE?$AA?$AA@ 0000000180001430     FARCmds.obj
 0001:00000440       ??_C@_19IJOJOJIB@?$AAP?$AAA?$AAT?$AAH?$AA?$AA@ 0000000180001440     FARCmds.obj
 0001:00000450       ??_C@_1O@PJHDHGJM@?$AAU?$AAn?$AAl?$AAo?$AAa?$AAd?$AA?$AA@ 0000000180001450     FARCmds.obj
 0001:00000460       ??_C@_1O@PAPHGGOK@?$AAU?$AAN?$AAL?$AAO?$AAA?$AAD?$AA?$AA@ 0000000180001460     FARCmds.obj
 0001:00000470       ??_C@_19OGNEHOBL@?$AAL?$AAo?$AAa?$AAd?$AA?$AA@ 0000000180001470     FARCmds.obj
 0001:00000480       ??_C@_19LIDMLGEF@?$AAL?$AAO?$AAA?$AAD?$AA?$AA@ 0000000180001480     FARCmds.obj
 0001:00000490       ??_C@_17NMIMIGP@?$AAR?$AAu?$AAn?$AA?$AA@ 0000000180001490     FARCmds.obj
 0001:00000498       ??_C@_17KKFGGCGH@?$AAR?$AAU?$AAN?$AA?$AA@ 0000000180001498     FARCmds.obj
 0001:000004a0       ??_C@_19IJIONFBP@?$AAL?$AAi?$AAn?$AAk?$AA?$AA@ 00000001800014a0     FARCmds.obj
 0001:000004b0       ??_C@_19NHGGBNEB@?$AAL?$AAI?$AAN?$AAK?$AA?$AA@ 00000001800014b0     FARCmds.obj
 0001:000004c0       ??_C@_19JKCOJBMF@?$AAG?$AAo?$AAt?$AAo?$AA?$AA@ 00000001800014c0     FARCmds.obj
 0001:000004d0       ??_C@_19MEMGFJJL@?$AAG?$AAO?$AAT?$AAO?$AA?$AA@ 00000001800014d0     FARCmds.obj
 0001:000004e0       ??_C@_19PLOBJMHF@?$AAE?$AAd?$AAi?$AAt?$AA?$AA@ 00000001800014e0     FARCmds.obj
 0001:000004f0       ??_C@_19KFAJFECL@?$AAE?$AAD?$AAI?$AAT?$AA?$AA@ 00000001800014f0     FARCmds.obj
 0001:00000500       ??_C@_1BA@BCPLKBBA@?$AAW?$AAh?$AAe?$AAr?$AAe?$AAI?$AAs?$AA?$AA@ 0000000180001500     FARCmds.obj
 0001:00000510       ??_C@_1BA@NBLHMMII@?$AAW?$AAH?$AAE?$AAR?$AAE?$AAI?$AAS?$AA?$AA@ 0000000180001510     FARCmds.obj
 0001:00000520       ??_C@_19KKHIGANA@?$AAC?$AAl?$AAi?$AAp?$AA?$AA@ 0000000180001520     FARCmds.obj
 0001:00000530       ??_C@_19PEJAKIIO@?$AAC?$AAL?$AAI?$AAP?$AA?$AA@ 0000000180001530     FARCmds.obj
 0001:00000540       ??_C@_1BC@ENICKDH@?$AAC?$AAo?$AAn?$AAt?$AAe?$AAn?$AAt?$AAs?$AA?$AA@ 0000000180001540     FARCmds.obj
 0001:00000558       ??_C@_19MJAKNMNK@?$AAV?$AAi?$AAe?$AAw?$AA?$AA@ 0000000180001558     FARCmds.obj
 0001:00000568       ??_C@_19JHOCBEIE@?$AAV?$AAI?$AAE?$AAW?$AA?$AA@ 0000000180001568     FARCmds.obj
 0001:00000578       ??_C@_17NACPPFBM@?$AAF?$AAA?$AAR?$AA?$AA@ 0000000180001578     FARCmds.obj
 0001:00000580       ??_C@_1DE@BGKMIKPD@?$AAE?$AAu?$AAg?$AAe?$AAn?$AAe?$AA?5?$AAR?$AAo?$AAs?$AAh?$AAa?$AAl?$AA?5?$AA?$CG?$AA?5?$AAF?$AAa?$AAr?$AA?5?$AAG?$AAr?$AAo?$AAu?$AAp?$AA?$AA@ 0000000180001580     FARCmds.obj
 0001:000005c0       ??_C@_1EI@IHKPBHMH@?$AAF?$AAA?$AAR?$AA?5?$AAC?$AAo?$AAm?$AAm?$AAa?$AAn?$AAd?$AAs?$AA?5?$AAP?$AAl?$AAu?$AAg?$AAi?$AAn?$AA?5?$AAf?$AAo?$AAr?$AA?5?$AAF?$AAa?$AAr?$AA?5?$AAM?$AAa?$AAn?$AAa@ 00000001800015c0     FARCmds.obj
 0001:00000608       ??_C@_1BA@LGNBLCFH@?$AAF?$AAA?$AAR?$AAC?$AAm?$AAd?$AAs?$AA?$AA@ 0000000180001608     FARCmds.obj
 0001:00000620       ??_C@_1GK@KLNCFMI@?$AAf?$AAa?$AAr?$AA?3?$AAv?$AAi?$AAe?$AAw?$AA?3?$AAe?$AAd?$AAi?$AAt?$AA?3?$AAg?$AAo?$AAt?$AAo?$AA?3?$AAc?$AAl?$AAi?$AAp?$AA?3?$AAw?$AAh?$AAe?$AAr?$AAe?$AAi?$AAs?$AA?3@ 0000000180001620     FARCmds.obj
 0001:00000690       ??_7?$DialogItemBinding@UFarDialogItem@@@@6B@ 0000000180001690     FARCmds.obj
 0001:000006a0       ??_7?$DialogBuilderBase@UFarDialogItem@@@@6B@ 00000001800016a0     FARCmds.obj
 0001:000006e8       ??_C@_15EFLNJKHH@?$AA?$CF?$AAu?$AA?$AA@ 00000001800016e8     FARCmds.obj
 0001:000006f0       ??_7PluginUIntEditFieldBinding@@6B@ 00000001800016f0     FARCmds.obj
 0001:00000700       ??_7PluginDialogBuilder@@6B@ 0000000180001700     FARCmds.obj
 0001:00000748       ??_7PluginCheckBoxBinding@@6B@ 0000000180001748     FARCmds.obj
 0001:00000758       ??_7PluginRadioButtonBinding@@6B@ 0000000180001758     FARCmds.obj
 0001:00000768       ??_7PluginIntEditFieldBinding@@6B@ 0000000180001768     FARCmds.obj
 0001:00000778       ??_C@_1O@BJPKKLLM@?$AAC?$AAo?$AAn?$AAf?$AAi?$AAg?$AA?$AA@ 0000000180001778     FARCmds.obj
 0001:000007a0       _alloca_probe              00000001800017a0     chkstk.obj
 0001:000007a0       __chkstk                   00000001800017a0 f   chkstk.obj
 0001:000007f0       ?GetLangString@PluginDialogBuilder@@MEAAPEB_WH@Z 00000001800017f0 f i FARCmds.obj
 0001:00000800       ?GetInt@@YAHPEA_W0@Z       0000000180001800 f   FARCmds.obj
 0001:00000870       ?PartCmdLine@@YAHPEB_WPEA_WH1H@Z 0000000180001870 f   FARCmds.obj
 0001:00000980       ?ProcessOSAliases@@YAHPEA_WH@Z 0000000180001980 f   FARCmds.obj
 0001:00000c70       ?isDevice@@YA_NPEB_W0@Z    0000000180001c70 f i FARCmds.obj
 0001:00001000       ?ThreadWhatUpdateScreen@@YAKPEAX@Z 0000000180002000 f   FARCmds.obj
 0001:000015b0       ?OpenFromCommandLine@@YAHPEB_W@Z 00000001800025b0 f   FARCmds.obj
 0001:00003260       GetGlobalInfoW             0000000180004260 f   FARCmds.obj
 0001:000032e0       SetStartupInfoW            00000001800042e0 f   FARCmds.obj
 0001:000035f0       OpenW                      00000001800045f0 f   FARCmds.obj
 0001:00003960       GetPluginInfoW             0000000180004960 f   FARCmds.obj
 0001:00003a40       ?InitDialogItem@?$DialogBuilderBase@UFarDialogItem@@@@MEAAXPEAUFarDialogItem@@PEB_W@Z 0000000180004a40 f i FARCmds.obj
 0001:00003a40       ?SaveValue@?$DialogItemBinding@UFarDialogItem@@@@UEAAXPEAUFarDialogItem@@H@Z 0000000180004a40 f i FARCmds.obj
 0001:00003a50       ?TextWidth@?$DialogBuilderBase@UFarDialogItem@@@@MEAAHAEBUFarDialogItem@@@Z 0000000180004a50 f i FARCmds.obj
 0001:00003a60       ?AddIntEditField@?$DialogBuilderBase@UFarDialogItem@@@@UEAAPEAUFarDialogItem@@PEAHH@Z 0000000180004a60 f i FARCmds.obj
 0001:00003a60       ?CreateCheckBoxBinding@?$DialogBuilderBase@UFarDialogItem@@@@MEAAPEAU?$DialogItemBinding@UFarDialogItem@@@@PEAHH@Z 0000000180004a60 f i FARCmds.obj
 0001:00003a60       ?AddUIntEditField@?$DialogBuilderBase@UFarDialogItem@@@@UEAAPEAUFarDialogItem@@PEAIH@Z 0000000180004a60 f i FARCmds.obj
 0001:00003a60       ?CreateRadioButtonBinding@?$DialogBuilderBase@UFarDialogItem@@@@MEAAPEAU?$DialogItemBinding@UFarDialogItem@@@@PEAH@Z 0000000180004a60 f i FARCmds.obj
 0001:00003a60       ?GetLangString@?$DialogBuilderBase@UFarDialogItem@@@@MEAAPEB_WH@Z 0000000180004a60 f i FARCmds.obj
 0001:00003a70       ?DoShowDialog@?$DialogBuilderBase@UFarDialogItem@@@@MEAA_JXZ 0000000180004a70 f i FARCmds.obj
 0001:00003a80       ??1?$DialogBuilderBase@UFarDialogItem@@@@MEAA@XZ 0000000180004a80 f i FARCmds.obj
 0001:00003b00       ??_E?$DialogBuilderBase@UFarDialogItem@@@@MEAAPEAXI@Z 0000000180004b00 f i FARCmds.obj
 0001:00003b00       ??_G?$DialogBuilderBase@UFarDialogItem@@@@MEAAPEAXI@Z 0000000180004b00 f i FARCmds.obj
 0001:00003b30       ?ReallocDialogItems@?$DialogBuilderBase@UFarDialogItem@@@@IEAAXXZ 0000000180004b30 f i FARCmds.obj
 0001:00003c50       ?ItemWidth@?$DialogBuilderBase@UFarDialogItem@@@@IEAA_JAEBUFarDialogItem@@@Z 0000000180004c50 f i FARCmds.obj
 0001:00003ce0       ?MaxTextWidth@?$DialogBuilderBase@UFarDialogItem@@@@IEAA_JXZ 0000000180004ce0 f i FARCmds.obj
 0001:00003e00       ??0PluginUIntEditFieldBinding@@QEAA@AEBUPluginStartupInfo@@PEAPEAXHPEAIH@Z 0000000180004e00 f i FARCmds.obj
 0001:00003ec0       ?SaveValue@PluginUIntEditFieldBinding@@UEAAXPEAUFarDialogItem@@H@Z 0000000180004ec0 f i FARCmds.obj
 0001:00003f10       ?InitDialogItem@PluginDialogBuilder@@MEAAXPEAUFarDialogItem@@PEB_W@Z 0000000180004f10 f i FARCmds.obj
 0001:00003f40       ?TextWidth@PluginDialogBuilder@@MEAAHAEBUFarDialogItem@@@Z 0000000180004f40 f i FARCmds.obj
 0001:00003f50       ?DoShowDialog@PluginDialogBuilder@@MEAA_JXZ 0000000180004f50 f i FARCmds.obj
 0001:00003ff0       ?SaveValue@PluginCheckBoxBinding@@UEAAXPEAUFarDialogItem@@H@Z 0000000180004ff0 f i FARCmds.obj
 0001:00004050       ?SaveValue@PluginRadioButtonBinding@@UEAAXPEAUFarDialogItem@@H@Z 0000000180005050 f i FARCmds.obj
 0001:000040a0       ??0PluginIntEditFieldBinding@@QEAA@AEBUPluginStartupInfo@@PEAPEAXHPEAHH@Z 00000001800050a0 f i FARCmds.obj
 0001:00004160       ?SaveValue@PluginIntEditFieldBinding@@UEAAXPEAUFarDialogItem@@H@Z 0000000180005160 f i FARCmds.obj
 0001:000041b0       ?CreateCheckBoxBinding@PluginDialogBuilder@@MEAAPEAU?$DialogItemBinding@UFarDialogItem@@@@PEAHH@Z 00000001800051b0 f i FARCmds.obj
 0001:00004230       ?CreateRadioButtonBinding@PluginDialogBuilder@@MEAAPEAU?$DialogItemBinding@UFarDialogItem@@@@PEAH@Z 0000000180005230 f i FARCmds.obj
 0001:000042a0       ??_EPluginDialogBuilder@@UEAAPEAXI@Z 00000001800052a0 f i FARCmds.obj
 0001:000042a0       ??_GPluginDialogBuilder@@UEAAPEAXI@Z 00000001800052a0 f i FARCmds.obj
 0001:000042f0       ?AddDialogItem@?$DialogBuilderBase@UFarDialogItem@@@@IEAAPEAUFarDialogItem@@W4FARDIALOGITEMTYPES@@PEB_W@Z 00000001800052f0 f i FARCmds.obj
 0001:00004380       ?AddRadioButtons@?$DialogBuilderBase@UFarDialogItem@@@@QEAAXPEAHHQEBH_N@Z 0000000180005380 f i FARCmds.obj
 0001:00004540       ?AddTextBefore@?$DialogBuilderBase@UFarDialogItem@@@@QEAAPEAUFarDialogItem@@PEAU2@H@Z 0000000180005540 f i FARCmds.obj
 0001:00004640       ?UpdateBorderSize@?$DialogBuilderBase@UFarDialogItem@@@@IEAAXXZ 0000000180005640 f i FARCmds.obj
 0001:00004700       ??_GPluginCheckBoxBinding@@UEAAPEAXI@Z 0000000180005700 f i FARCmds.obj
 0001:00004700       ??_GPluginRadioButtonBinding@@UEAAPEAXI@Z 0000000180005700 f i FARCmds.obj
 0001:00004700       ??_G?$DialogItemBinding@UFarDialogItem@@@@UEAAPEAXI@Z 0000000180005700 f i FARCmds.obj
 0001:00004700       ??_GPluginUIntEditFieldBinding@@UEAAPEAXI@Z 0000000180005700 f i FARCmds.obj
 0001:00004700       ??_EPluginIntEditFieldBinding@@UEAAPEAXI@Z 0000000180005700 f i FARCmds.obj
 0001:00004700       ??_EPluginUIntEditFieldBinding@@UEAAPEAXI@Z 0000000180005700 f i FARCmds.obj
 0001:00004700       ??_EPluginRadioButtonBinding@@UEAAPEAXI@Z 0000000180005700 f i FARCmds.obj
 0001:00004700       ??_GPluginIntEditFieldBinding@@UEAAPEAXI@Z 0000000180005700 f i FARCmds.obj
 0001:00004700       ??_EPluginCheckBoxBinding@@UEAAPEAXI@Z 0000000180005700 f i FARCmds.obj
 0001:00004700       ??_E?$DialogItemBinding@UFarDialogItem@@@@UEAAPEAXI@Z 0000000180005700 f i FARCmds.obj
 0001:00004730       ?AddIntEditField@PluginDialogBuilder@@UEAAPEAUFarDialogItem@@PEAHH@Z 0000000180005730 f i FARCmds.obj
 0001:00004840       ?AddUIntEditField@PluginDialogBuilder@@UEAAPEAUFarDialogItem@@PEAIH@Z 0000000180005840 f i FARCmds.obj
 0001:00004950       ConfigureW                 0000000180005950 f   FARCmds.obj
 0001:000057e0       wcschr                     00000001800067e0 f   libCRT64:strchr.obj
 0001:00005800       wcsstr                     0000000180006800 f   libCRT64:strstr.obj
 0001:00005870       memcpy                     0000000180006870 f   libCRT64:memcpy.obj
 0001:000058a0       memmove                    00000001800068a0 f   libCRT64:memmove.obj
 0001:00005900       _memicmp                   0000000180006900 f   libCRT64:memicmp.obj
 0001:00005970       memcmp                     0000000180006970 f   libCRT64:memcmp.obj
 0001:000059a0       ??_V@YAXPEAX@Z             00000001800069a0 f   libCRT64:delete_array.obj
 0001:000059b0       ??_U@YAPEAX_K@Z            00000001800069b0 f   libCRT64:new_array.obj
 0001:000059c0       swab                       00000001800069c0 f   libCRT64:swab.obj
 0001:00005a20       free                       0000000180006a20 f   libCRT64:free.obj
 0001:00005a50       malloc                     0000000180006a50 f   libCRT64:malloc.obj
 0001:00005a80       memset                     0000000180006a80 f   libCRT64:memset.obj
 0001:00005ab0       ??3@YAXPEAX@Z              0000000180006ab0 f   libCRT64:delete.obj
 0001:00005ac0       ??2@YAPEAX_K@Z             0000000180006ac0 f   libCRT64:new.obj
 0001:00005eb4       __IMPORT_DESCRIPTOR_KERNEL32 0000000180006eb4     kernel32:KERNEL32.dll
 0001:00005ec8       __IMPORT_DESCRIPTOR_ADVAPI32 0000000180006ec8     advapi32:ADVAPI32.dll
 0001:00005edc       __NULL_IMPORT_DESCRIPTOR   0000000180006edc     kernel32:KERNEL32.dll
 0002:00000000       ?OptName@@3UOptionsName@@A 0000000180008000     FARCmds.obj
 0002:00000170       ?cmd@@3PA_WA               0000000180008170     FARCmds.obj
 0002:00000b98       ?Opt@@3UOptions@@A         0000000180008b98     FARCmds.obj
 0002:00000bc0       ?fullcmd@@3PA_WA           0000000180008bc0     FARCmds.obj
 0002:000015f0       ?selectItem@@3PA_WA        00000001800095f0     FARCmds.obj
 0002:00002020       ?PInfo@@3UPanelInfo@@A     000000018000a020     FARCmds.obj

 entry point at        0000:00000000

 Static symbols

 0001:00000d00       ?validForView@@YA_NPEB_WHH@Z 0000000180001d00 f   FARCmds.obj
 0001:00000f50       ?showPartOfOutput@@YAKPEAUTShowOutputStreamData@@@Z 0000000180001f50 f   FARCmds.obj
 0001:000011d0       ?loadFile@@YAPEA_WPEB_WKHAEA_KAEA_N@Z 00000001800021d0 f   FARCmds.obj
 0001:00001470       ?ParseCmdSyntax@@YAXAEAPEA_WAEAH1@Z 0000000180002470 f   FARCmds.obj
